:0200000480007A
:100000006F008004732F2034930F80006308FF0378
:10001000930F90006304FF03930FB0006300FF038E
:10002000130F000063040F0067000F00732F2034CC
:1000300063540F006F00400093E19153171F0000BD
:1000400023223FFC6FF09FFF93000000130100008C
:10005000930100001302000093020000130300004C
:100060009303000013040000930400001305000034
:10007000930500001306000093060000130700001C
:100080009307000013080000930800001309000004
:1000900093090000130A0000930A0000130B0000EC
:1000A000930B0000130C0000930C0000130D0000D4
:1000B000930D0000130E0000930E0000130F0000BC
:1000C000930F0000732540F16310050097020000B4
:1000D000938202017390523073500018970200000F
:1000E00093824202739052309B021000939252030B
:1000F0009382F2FF7390023B9302F0017390023AF5
:100100007350403097020000938242017390523046
:10011000735020307350303093010000970200007C
:10012000938282EE73905230130510001315F5017F
:10013000635C05000F00F00F930110009308D005D9
:10014000130500007300000093020000638A0200A0
:1001500073905210B7B200009B82921073902230BD
:100160007350003097020000938242017390123462
:10017000732540F1730020309301200093020000AA
:100180001703000013030301E70203006F00000ED2
:10019000170300001303C3FF639A620C930130003E
:1001A0009702000093820201E78202006F00000CB8
:1001B000170300001303C3FF639A620A9301400010
:1001C000130200001703000013030301E7060300F6
:1001D000631E30081302120093022000E31452FE43
:1001E00093015000130200001703000013034301A2
:1001F00013000000E7060300631A30061302120022
:1002000093022000E31252FE9301600013020000EB
:100210001703000013038301130000001300000004
:10022000E706030063143004130212009302200057
:10023000E31052FE93021000170300001303C301E2
:100240006700C3FF93821200938212009382120010
:100250009382120093821200938212009303400053
:100260009301700063947200631030020F00F00F6E
:10027000638001009391110093E111009308D00570
:1002800013850100730000000F00F00F93011000B0
:100290009308D0051305000073000000731000C020
:1002A000000000000000000000000000000000004E
:0C02B00000000000000000000000000042
:1010000000000000000000000000000000000000E0
:1010100000000000000000000000000000000000D0
:1010200000000000000000000000000000000000C0
:1010300000000000000000000000000000000000B0
:081040000000000000000000A8
:040000058000000077
:00000001FF
